S025000062696E2F64656D6F70726F675F6F6C696D65785F65666D3332673838302E737265634A
S113200070040020412400003D2200003D22000015
S11320103D2200003D2200003D2200003D22000040
S11320203D2200003D2200003D2200003D22000030
S11320303D2200003D2200003D2200003D2500001D
S11320403D2200003D2200003D2200003D22000010
S11320503D2200003D2200003D2200003D22000000
S11320603D2200003D2200003D2200003D220000F0
S11320703D2200003D2200003D2200003D220000E0
S11320803D2200003D2200003D2200003D220000D0
S11320903D2200003D2200003D2200003D220000C0
S11320A03D2200003D2200003D220000952D00004D
S11320B03D2200003D220000EE11AA5570B584B007
S11320C01E4B0FCB8DE80F0001211D4800F0D4FBFF
S11320D0012304220621022000F086FD00230122B0
S11320E00721022000F080FD0121164800F0C4FB06
S11320F00221154800F00EFD144C0121204600F089
S113210013FB0121204600F0B7FB00268DF8006088
S11321100F4C6946204600F059FA4FF416523146E6
S1132120204600F013FA0323636504236363052147
S1132130204600F031FA04B070BD00BFB82F000093
S113214000C2020000230400030012004015160020
S113215000440840074BDB6A13F0040F07D010B5A6
S11321600446044800F05AFA2070012010BD0020F3
S1132170704700BF0044084008B5FFF79FFF08BD43
S1132180BFF34F8F0449CA6802F4E062034B134360
S1132190CB60BFF34F8FFEE700ED00E00400FA05CB
S11321A008B5204B1B789BB91F48FFF7D3FF0128C4
S11321B036D11D4B1B78002B32D000F0B9F91B4BE4
S11321C018600122174B1A700022194B1A7008BDAF
S11321D0174B1B78013314481844FFF7BBFF012841
S11321E014D1134A13780133DBB213700E4A1278F8
S11321F0934215D100220B4B1A700B4B5B78FF2BCB
S11322000ED1094B9B785BB9FFF7BAFF00F090F948
S1132210064B1B686433984202D90022014B1A70A2
S113222008BD00BF5100002010000020080000205D
S11322300C00002008B5FFF7B3FF08BDFEE700BFA0
S113224000B583B000F0A0FE5E4B1B681B0E0DD1E1
S11322505D490A6822F070020A605C4A116821F044
S113226060411160116861F060611160032B11D845
S1132270564A136823F4FC531360002302F50052FA
S11322802032136004321360143213600832136076
S11322901832136001A800F0C9F99DF80430012B2D
S11322A010D19DF8053023B9494A136843F002035D
S11322B013609DF80530012B04D8464A136843F097
S11322C001031360444B1A68444B9A4221D8414994
S11322D00B6843F490430B60414803681B0A1B06D8
S11322E003F0FE4203681B0403F4FE031343026875
S11322F002F4FE421343026802F07F021343394A98
S11323001360394B1A68394B1A600B6823F49043F5
S11323100B6001221146002000F0D4FB344A136CF8
S113232043F00F031364536C6FEA13436FEA0343E0
S1132330536400212F4800F09FFA00212E4800F03A
S11323409BFA00212D4800F097FA00212C4800F058
S113235093FA00212B4800F08FFA00212A4800F05C
S11323608BFA0021294800F087FA0021284800F060
S113237083FA0021274800F07FFA0021264800F064
S11323807BFA0021254800F077FA0021244800F068
S113239073FA0021234800F06FFA0021224800F06C
S11323A06BFA012305220921184600F01DFC0221C5
S11323B0012000F009FC00F069F800F09BF803B07C
S11323C05DF804FBFC81E00F0CA00C4020600C4085
S11323D040800C4044800C40F081E00FFFB98A4CEF
S11323E0B481E00F34200040C881E00F2C4000404D
S11323F000800C40000304000013040000330400B8
S113240000A20200000202000012020000220200E8
S113241000320200007202000082020000B20200D8
S113242000E2020000F2020000D2020008B5FFF749
S113243007FFFFF7A1FE00F031F8FFF7FBFEFAE714
S113244008B50F498D460B4B0B4A03E01168196020
S11324500433043209498B42F8D30A480A494FF03D
S113246000028842B8BF40F8042BFADBFFF7DEFF16
S113247008BD00BF00000020CC2F00000800002091
S113248070040020080000207000002008B50248F5
S113249000F0D6FC08BD00BF00A0084010B500F055
S11324A047F80E4B1B68C31AB3F5FA7F14D30446DE
S11324B00B4B1B783BB90122094B1A7000210948C8
S11324C000F084FC06E00021054B19700A4605481B
S11324D000F07CFC014B1C6010BD00BF54000020C8
S11324E05800002000A00840014B1860704700BF4E
S11324F05C00002008B50A4800F058FA094BA3FB19
S1132500003080090138084B5860E021074A82F8FE
S113251023100020986007221A60FFF7E5FF08BD2A
S113252020000400D34D621010E000E000ED00E054
S1132530014B1868704700BF5C000020024A136812
S113254001331360704700BF5C00002038B50446B7
S11325501546084659B90D4B9C4205D003F58063D6
S11325609C4212D10A4800E00A4800F01FFA4201D6
S1132570B2FBF5F2203AD200236C13F0010F03D121
S1132580636C13F0040FFBD1E26038BD00400840D7
S11325904015160040051400CB435B0003F00A030A
S11325A01943036C13F0010F03D1436C13F0020FB2
S11325B0FBD14160704700BF29B1436C002BFCD1B3
S11325C001230364704700230364704738B504464D
S11325D00D46036C13F0010F03D1636C13F0020F6B
S11325E0FBD10A23636001212046FFF7E5FF22683F
S11325F022F01C022B7B1A436B7B1A43AB7B1343E5
S11326002360AA6869682046FFF7A0FF2B786360FF
S113261000212046FFF7D0FF38BD00BF836813F0C8
S1132620200FFBD0C069C0B2704700BF06490B69D8
S113263003F03F0303708B6903F0F002CB69C3F32B
S11326400313134343707047D0FF0FE00A4B5B68DA
S113265003F00702032A0CD8DFE802F0020207079E
S113266023F0070343F0010303E023F0070343F0DF
S11326700303014A5360704700000C40B0FA80F035
S1132680C0B2C0F11F007047134B5B68134A024489
S113269013498A420DD803F00702023A012A04D8EA
S11326A023F0070343F0030303E023F0070343F09D
S11326B001030C4A90420BD803F00702023A012AA4
S11326C004D823F0070343F0020301E023F00703D7
S11326D0014A5360704700BF00000C40FFDB0BFF52
S11326E0FF23F4000024F40000487047809FD500C5
S11326F008B50C4B9B6A400023FA00F000F003007D
S1132700022806D0032807D0012809D100F03EFC96
S113271008BD00F03FFC08BD00F026FC400808BDE1
S1132720002008BD00800C4010B50C46C0F3031314
S1132730013B032B00F29880DFE803F0020C1C66D7
S11327400846FFF79BFF494A936823F00F03184399
S1132750906010BDFFF77AFF2046FFF78FFF434AD2
S1132760536823F00F031843506000F0FDFBFFF79C
S11327708BFF10BD3E4B98421BD003F5F6339842B5
S11327802CD0A3F57F3398426ED1384B5B6D13F098
S1132790010F04D1354B1B6D13F0040FFAD1204601
S11327A0FFF76CFF314A936E23F00F0318439066D2
S11327B010BD2E4B5B6D13F0010F04D12B4B1B6D21
S11327C013F0040FFAD12046FFF758FF274A936EFF
S11327D023F0F00343EA0010906610BD234B5B6DB9
S11327E013F0010F04D1214B1B6D13F0040FFAD128
S11327F02046FFF743FF1D4A936E23F440731038BD
S113280043EA0023936610BD1A4B984204D003F5A3
S11328100433984214D010BD144B5B6D13F0010FB8
S113282004D1124B1B6D13F0400FFAD12046FFF771
S113283025FF0E4A136F23F003031843106710BDDE
S11328400A4B5B6D13F0010F04D1084B1B6D13F0A1
S1132850400FFAD12046FFF711FF044A136F23F00B
S1132860300343EA0010106710BD00BF00800C4025
S113287030140A004005140010B4C0F30323013BD4
S1132880052B27D8DFE803F0031206090C0F0022FA
S1132890114C0DE00022114C0AE00122104C07E01B
S11328A01022104C04E000220F4C01E000220F4CD7
S11328B0C0F3043042B10E4B5B6D13F0010F03D132
S11328C00B4B1B6D1A42FBD104F1047400EBC400E2
S11328D08000016010BC704708800C4040800C40B0
S11328E058800C4060800C4078800C4044800C4040
S11328F000800C4000F00F000138032839D8DFE8CD
S113290000F004182802072070471E4BDB6A03F40A
S11329107053B3F5805F2ED0B3F5005F03D0B3F5E9
S1132920006F04D101E002207047042070470520A5
S11329307047144B9B6A03F00303022B1DD0032B37
S113294003D0012B03D103207047062070470120D8
S113295070470C4B9B6A03F00C03022B0FD0032B24
S113296003D0012B03D103207047062070470120B8
S113297070470020704703207047022070470220F0
S1132980704700BF00800C4008B50748FFF7B2FF4E
S1132990072804D0082805D100F098FA08BDFFF7ED
S11329A0A3FE08BD002008BD0400180008B500F40B
S11329B07810B0F5402F4CD012D8B0F5802F2FD01E
S11329C004D810B3B0F5003F22D076E0B0F5002F64
S11329D02DD0B0F5202F33D0B0F5C02F6DD122E02B
S11329E0B0F5A01F51D006D8B0F5602F3AD0B0F59D
S11329F0901F46D061E0B0F5C01F58D0B0F5D01F8D
S1132A0058D0B0F5B01F58D148E000F05FFA08BDC7
S1132A1000F05CFA2A4B9B6803F00F03D84008BD12
S1132A2000F0A2FA08BD0020FFF762FE08BD0020F6
S1132A30FFF75EFE224B9B6E03F00F03D84008BDE8
S1132A400020FFF755FE1E4B9B6EC3F30313D840C3
S1132A5008BD0020FFF74CFE194B9B6EC3F3012306
S1132A60D84008BD0020FFF743FE154A936EC3F318
S1132A700123D840D36F03F007030133B0FBF3F015
S1132A8008BD0120FFF734FE08BD0120FFF730FE2A
S1132A900B4B1B6F03F00303D84008BD0120FFF765
S1132AA027FE074B1B6FC3F30113D84008BDFFF784
S1132AB06BFF08BDFFF718FE08BD002008BD00BF6E
S1132AC000800C4008B5042821D8DFE800F00C0988
S1132AD011030600012302200CE01023202009E04A
S1132AE04023802006E04FF480734FF4007001E02F
S1132AF00423082039B106490B6232B1044BDB6A66
S1132B001842FBD001E0024B186200F0D1F808BD76
S1132B1000800C4010B500F00F00012804D00028FC
S1132B204DD0032821D910BD0239032947D8DFE845
S1132B3001F0020B05080020042407E002200446EB
S1132B4004E00320012401E00120032401221146B2
S1132B50FFF7B8FFFFF77AFD194B5C6200F0A8F8A5
S1132B6000F002FAFFF790FD10BD022801D1002405
S1132B7000E002240139052921D8DFE801F0160319
S1132B800A202011012211460020FFF79BFF022397
S1132B900CE0012211461046FFF794FF012305E0E3
S1132BA00122084B1A60032300E000230448816AD1
S1132BB00322A24021EA0202A3401343836210BD10
S1132BC000800C400808904330B4064AC40025181D
S1132BD0AB001D46D35823F003031943515130BCB5
S1132BE0704700BF00600040F0B51446AAB153B16D
S1132BF001258D4000EBC006B20002F1804202F5CF
S1132C00C042156109E001258D4000EBC006B20009
S1132C1002F1804202F5C0425561072915D8DFF858
S1132C208CC0C7003D18AA00624456684FEA810E62
S1132C300F2202FA0EF226EA020504FA0EF22A43E1
S1132C403D18AE006644726015E0DFF860E0C7002E
S1132C503D18AA007244966801F18042083A920035
S1132C600F25954026EA050504FA02F22A433D1889
S1132C70AE007644B260BCB95BB1012303FA01F142
S1132C8000EBC000830003F1804303F5C0431961E6
S1132C90F0BD012303FA01F100EBC000830003F14E
S1132CA0804303F5C0435961F0BD00BF006000409C
S1132CB0024BDA6A024B1A80704700BF00800C4056
S1132CC0600000201F2A01DD203A0431012303FAA9
S1132CD002F2072924D8DFE801F004080C101418C4
S1132CE01C20036C1A4302647047436C1A43426409
S1132CF07047836C1A4382647047C36C1A43C2647E
S1132D007047036D1A4302657047436D1A43426569
S1132D107047836D1A4382657047C36D1A43C26559
S1132D20704700BF1F2A01DD203A0431012303FA52
S1132D3002F207292CD8DFE801F004090E13181D4C
S1132D402227036C23EA020202647047436C23EADD
S1132D50020242647047836C23EA02028264704771
S1132D60C36C23EA0202C2647047036D23EA0202C1
S1132D7002657047436D23EA020242657047836D22
S1132D8023EA020282657047C36D23EA0202C26528
S1132D90704700BF4FF0FF32034B5A62034A136877
S1132DA001331360704700BF00A008406400002096
S1132DB00023036403654364436583648365C364D8
S1132DC0C365436E002BFCD1704700BF10B50B29BF
S1132DD02AD8DFE801F02706090C0F1215181B1E6C
S1132DE02124032301241FE003231C461CE00323A6
S1132DF0002419E00323022416E02723002413E00F
S1132E002723032410E0012303240DE001230224DB
S1132E100AE001231C4607E001231C4604E00723C3
S1132E20032401E00F23032422B11A462146FFF7AD
S1132E3049FF10BD1A462146FFF774FF10BD00BFBD
S1132E4010B504461E4B9A6A22F003029A629A6AEB
S1132E5042F002029A629A6D42F004029A659A6EF6
S1132E6022F440729A669A6E42F440729A66002383
S1132E708362636E002BFCD14FF0FF3363624FF02B
S1132E800062104B1A600123A36241F60B73636066
S1132E9000220B4BDA672046FFF78AFF40F2FF332C
S1132EA0A36005232360636E002BFCD1064BE36013
S1132EB0636E002BFCD101236362A36210BD00BFCB
S1132EC000800C4000E100E000011C001D4BDB6AA7
S1132ED003F47053B3F5805F2FD0B3F5005F03D0D4
S1132EE0B3F5006F06D102E0174B18687047174B13
S1132EF018687047134BDB6803F4E063B3F5007F95
S1132F0013D004D8ABB1B3F5807F10D013E0B3F580
S1132F10806F15D0B3F5A06F03D0B3F5407F0AD10D
S1132F2001E00B4870470B4870470B4870470B484B
S1132F3070470B487047002070474FF400407047BB
S1132F400848704700800C40000000200400002066
S1132F50003FAB01809FD500C0D8A700C0CF6A0056
S1132F6040420F00406F400108B5FFF7AFFF044B2C
S1132F705B6803F00F03D840024B186008BD00BF24
S1132F8000800C4068000020704700BF4FF40040F0
S1132F90704700BF014B1868704700BF0000002055
S1132FA0F8B500BFF8BC08BC9E467047F8B500BF32
S1132FB0F8BC08BC9E4670470500000000000000F5
S10F2FC08025000000000000000000005C
S10B2FCC008000000048E80148
S9032000DC
